:020000020000FC
:0200000013C02B
:02001A003FC0E5
:1000260021C00FED0DBF0FEF07BB00E008BB0FE7C8
:1000360001BB00E002BB01E00ABB02E00BBB02E031
:1000460000BF03E003BF05ED06BF01E009BF08E0FE
:100056000BBF02E004B900E305BF00E808B97894D5
:100066008895FECF29B3209521FD02C000E002BF8E
:1000760021FF0DC002B7033050F0053310F013D046
:10008600432F330F639502B70D3008F0339500E226
:1000960005BF189508D033274FEF552700E002BF5C
:1000A60000E305BF1895693029F4431709F405D014
:1000B60066270895332766270895503009F07FC0D4
:1000C600032F02950F70132F10951F70011709F05B
:1000D60076C01127E2E7F0E0E00FF11F09940FC0A8
:1000E60014C019C01EC023C028C02DC032C037C0DE
:1000F6003CC041C046C04BC050C055C05AC008B3F2
:1001060000FDC09800FFC09A5AC008B301FDC1980F
:1001160001FFC19A54C008B302FDC29802FFC29AF9
:100126004EC008B303FDC39803FFC39A48C008B383
:1001360004FDC49804FFC49A42C008B305FDC598DF
:1001460005FFC59A3CC008B306FDC69806FFC69AC9
:1001560036C008B307FDC79807FFC79A30C002B379
:1001660000FD909800FF909A2AC002B301FD919875
:1001760001FF919A24C002B302FD929802FF929A5F
:100186001EC002B303FD939803FF939A18C002B3EF
:1001960004FD949804FF949A12C002B305FD959845
:1001A60005FF959A0CC002B306FD969806FF969A2F
:1001B60006C00BB300FDD89800FFD89A00C051E0E6
:0201C60008959A
:00000001FF
